:1000000000308A000428000084011F308305831615
:100010001F08F0399F0083121F1307309F008501CE
:1000200083161F080F399F0083121F080C399F0089
:100030000830A000A01D24280730810181308400F1
:100040000008C0390F388000640081308400000847
:10005000C03920048000900100306500073099000D
:100060008316050810308312A000A00B352800006D
:1000700019088C11051464006400640064006400B5
:100080006400640064006400640064006400640050
:100090006400640064006400640064006400640040
:1000A000640064000510640064006400640064007F
:1000B0006400640064006400640064006400640020
:1000C0006400640064006400640064006400640010
:0A00D0006400640064003A28630035
:02400E00CB39AC
:00000001FF
